:020000040000FA
:0600000087EF14F012006E
:0600080086EF11F012006A
:06001800D1EF11F012000F
:0E10000001002C2900009800000009000000EB
:02100E00D9CF38
:10101000E6FFE1CFD9FFE652A0940F015F6B626A51
:10102000536B010EE66EE66AE66A540EE66E0F0E2C
:10103000E66E5DEC14F00B6E050EE15E0B50160EC5
:10104000616E0F019F0E5B6F7B0E606EDF6ADF507B
:101050000B6E0C6A080E0B5C000E0C5810E2DF5091
:10106000040DF3CFE9FFF4CFEAFF000EE926020EEC
:10107000EA22EE6AEE6AEE6AEE6ADF2AE8D7648C4C
:101080000F015C6B6498649C62A607D062960001B5
:10109000736B786B796B7A6BF7D70001010E8A6FEF
:1010A0008B6F8C6B8D6B806BDF6A020EDF5C26E2D0
:1010B000EA6ADF34FE0BEA36E96E6B0EE926000EB3
:1010C000EA22EE6AED6AEA6ADF34FE0BEA36E96E7E
:1010D000670EE926000EEA22EE6AED6ADF50EA6A40
:1010E000840FE96E000EEA22EF6ADF50EA6A860F8B
:1010F000E96E000EEA22EF6ADF2AD7D70001080E58
:101100006B6F020E6C6F0F01160E536F0201200EF3
:10111000026F020E036F080E016F840E006F000154
:10112000616B606BE552E552E7CFD9FF1200D9CF72
:10113000E6FFE1CFD9FFE6520001600507E164BA9E
:1011400005D0626A60806088020E606F6250040B96
:1011500006E06050040B03E06294ABEC0EF064A276
:1011600002D0A19498D06250010B09E06050010BAD
:1011700006E04DDFA0840001040E606F62906250B3
:10118000100B06E06050100B03E096EC0EF0629836
:1011900062AC19D060AC0FD0010EE66EE66A000EAC
:1011A000E66EE66A730EE66EE66A06EC13F00B6E08
:1011B000060EE15E0B50629C0001885101E0880739
:1011C000885101E10DDA6250200B05E06050200BE0
:1011D00002E07CEC0EF06250020B14E06050020B57
:1011E00011E0010EE66EE66A000EE66EE66AE6685B
:1011F0007F0EE66E06EC13F00B6E060EE15E0B50F2
:101200000F015F6B040E0001E76E6019E8AE02D0BB
:10121000E73402D0E750605D02E2A1943CD060A6C2
:1012200039D0DF6A040EDF5C35E262A632D063CFCC
:1012300081F000018151780BE842E842E842826F78
:10124000629681B508D08251EA6A860FE96E000E77
:10125000EA22EF7007D08251EA6A840FE96E000E2D
:10126000EA22EF70825103E1C2EC0EF010D0000EC2
:10127000E66EE66A810EE66E000EE66E720EE66EB1
:10128000E66A06EC13F00B6E060EE15E0B50DF2AE9
:10129000C9D700D0A194E552E552E7CFD9FF12009B
:1012A000D9CFE6FFE1CFD9FF020EE126FD0EDBA488
:1012B00007D0E66AFE0EDBCFE6FF23DAE552E55201
:1012C000FD0EDBA208D0010EE66EFE0EDBCFE6FFC0
:1012D00018DAE552E552FE0EDB500C6A530F0B6E26
:1012E0000F0E0C220BC0DEFF0CC0DDFFDECFE9FFCE
:1012F000DDCFEAFFFD0EDBCFEFFF020EE15C02E285
:10130000E16AE552E16EE552E7CFD9FF1200D9CF8D
:10131000E6FFE1CFD9FF020EE126FD0EDB500FE024
:10132000FE0EEA6ADB34FE0BEA36E96E6B0EE92646
:10133000000EEA22EECFDEFFEDCFDDFF0ED0FE0E77
:10134000EA6ADB34FE0BEA36E96E670EE926000E28
:10135000EA22EECFDEFFEDCFDDFFD9CFE9FFDACF16
:10136000EAFFEE50ED1003E1F36AF46A49D0DECFF4
:10137000E9FFDDCFEAFF020EE926000EEA22FB0EAE
:10138000DBCFEEFFFC0EDBCFEDFFDECFE9FFDDCFE5
:10139000EAFFEE52FA0EDBCFEFFF400E0B6EDECF10
:1013A000E9FFDDCFEAFF0B50EF16880E0B6EDECFA4
:1013B000E9FFDDCFEAFF0B50EF12FD0EDB500CE032
:1013C000FE0EEA6ADB34FE0BEA36E96E6B0EE926A6
:1013D000000EEA22EF740BD0FE0EEA6ADB34FE0B3D
:1013E000EA36E96E670EE926000EEA22EF74DECFD8
:1013F0000BF0DDCF0CF00BC0F3FF0CC0F4FF00D0FE
:10140000020EE15C02E2E16AE552E16EE552E7CFED
:10141000D9FF1200D9CFE6FFE1CFD9FF020EE126B6
:10142000FE0EDB5020E165C0E9FF66C0EAFFEE5228
:10143000080EEF6E65C0E9FF66C0EAFF020EE926FE
:10144000000EEA22200EEE6E020EED6E65C0E9FF80
:1014500066C0EAFF8C0EEF6E6BC0E9FF6CC0EAFF5E
:10146000840EEF6E3DD0FD0EDB50E8240D6EFE0EB7
:10147000DB50040DF3500D24040DF3CF0BF0F4CF2B
:101480000CF0000E0B26020E0C220BC0DEFF0CC06F
:10149000DDFF840E0B6EDECFE9FFDDCFEAFF0B50E0
:1014A000EF12FD0EDB50E8240D6EFE0EDB50040D36
:1014B000F3500D24010F040DF3CF0BF0F4CF0CF01B
:1014C000000E0B26020E0C220BC0DEFF0CC0DDFF4F
:1014D000840E0B6EDECFE9FFDDCFEAFF0B50EF127B
:1014E000020EE15C02E2E16AE552E16EE552E7CF0D
:1014F000D9FF1200D9CFE6FFE1CFD9FF64A84ED0C3
:10150000FE0EEA6ADB34FE0BEA36E96E6B0EE92664
:10151000000EEA22EE50EFCFEAFFE96E400EEE1623
:10152000EE6AEE6AEE6AFE0EEA6ADB34FE0BEA361B
:10153000E96E6B0EE926000EEA22EE50EFCFEAFFCD
:10154000E96EEE7CFE0EEA6ADB34FE0BEA36E96EEB
:101550006B0EE926000EEA22EF74400E0B6EFE0EB3
:10156000EA6ADB34FE0BEA36E96E6B0EE926000E02
:10157000EA22EE50EFCFEAFFE96E0B50EF16FE0EB7
:10158000EA6ADB34FE0BEA36E96E6B0EE926000EE2
:10159000EA22EE50EFCFEAFFE96EEF7CE552E7CFAB
:1015A000D9FF1200646A606A0001606B00D012000B
:1015B0000001605114E1646A606A160E616E0F01E9
:1015C0009F0E5B6F7B0E606ED08EA284A084F28E25
:1015D00064B602D06486FCD70001010E606F120071
:1015E00000018A514DE1010E8A6F8B5149E1010ED4
:1015F0008B6F020E705D0DE16BC0E9FF6CC0EAFFFE
:10160000EE52EF6A6BC0E9FF6CC0EAFFC80EEF6EE6
:1016100037D0700535E1836B63C0E9FF64C0EAFF32
:10162000EE52080EEF6E63C0E9FF64C0EAFF020EDF
:10163000E926000EEA22200EEE6E020EED6E63C069
:10164000E9FF64C0EAFF840EEF6E010E836F65C090
:10165000E9FF66C0EAFFEE52080EEF6E65C0E9FFD3
:1016600066C0EAFF020EE926000EEA22200EEE6EA8
:10167000020EED6E65C0E9FF66C0EAFF800EEF6EF8
:10168000120000018C6B8D6B020E705D1AE165C05B
:10169000E9FF66C0EAFFEE52080EEF6E65C0E9FF93
:1016A00066C0EAFF020EE926000EEA22280EEE6E60
:1016B000020EED6E65C0E9FF66C0EAFFC80EEF6E70
:1016C0001FD074510201265D000175510201275996
:1016D00004E226C274F027C275F0D1D86BC0E9FFCE
:1016E0006CC0EAFF020EE926000EEA22280EEE6E1A
:1016F000020EED6E6BC0E9FF6CC0EAFFC80EEF6E24
:101700001200D9CFE6FFE1CFD9FF020EE126000E8D
:10171000DE6E020EDD6EFD0EDB50E8240D6EFE0E59
:10172000DB50040DF3500D24040DF3CF0BF0F4CF78
:101730000CF0D9CFE9FFDACFEAFF0B50EE260C50C0
:10174000ED22DECFE9FFDDCFEAFFEF9EFD0EDB509D
:101750000FE1FE0EEA6ADB34FE0BEA36E96E670E35
:10176000E926000EEA22DECFEEFFDDCFEDFF0ED040
:10177000FE0EEA6ADB34FE0BEA36E96E6B0EE926F2
:10178000000EEA22DECFEEFFDDCFEDFFDECFE9FF78
:10179000DDCFEAFFEF9CDECFE9FFDDCFEAFF040EED
:1017A000E926000EEA22EF8C020EE15C02E2E16A19
:1017B000E552E16EE552E7CFD9FF120064980001CF
:1017C00073BF2BD078AF09D0020E706F8D5101E13D
:1017D00058DF00018B6B8A6B1FD065C0E9FF66C0C4
:1017E000EAFFEE52080EEF6E65C0E9FF66C0EAFF41
:1017F000020EE926000EEA22200EEE6E020EED6EBB
:1018000065C0E9FF66C0EAFF8C0EEF6E6BC0E9FFB2
:101810006CC0EAFF840EEF6E31D0020120AF0DD014
:101820000001010E706F8C5101E12BDF00018B6B09
:101830008A6B895101E1D4DE21D00001020E706F64
:1018400065C0E9FF66C0EAFFEE52080EEF6E65C0A4
:10185000E9FF66C0EAFF020EE926000EEA22200E2A
:10186000EE6E020EED6E65C0E9FF66C0EAFF840E03
:10187000EF6E8B6B8A6B895101E1B2DE1200D9CF1A
:10188000E6FFE1CFD9FFE652080EDF6E0001745D7E
:10189000000E75590BE274C0DFFF6F5103E1010EBA
:1018A0006F6F04D06F0502E1020E6F6FDF500B6E99
:1018B0000C6A0B50745D746F0C507559756F6BC06A
:1018C000E9FF6CC0EAFFEE52DFCFEFFF280E7D6F1D
:1018D000020E7E6F73B119D0DF5016E071C0F6FFB3
:1018E00072C0F7FF712B000E72230800F550E66EF0
:1018F0007DC0E9FF7EC0EAFF7D2B000E7E23E5520E
:10190000E750EF6EDF06E8D717D0DF5015E071C063
:10191000E9FF72C0EAFF712B000E7223EF50E66EF2
:101920007DC0E9FF7EC0EAFF7D2B000E7E23E552DD
:10193000E750EF6EDF06E9D7E552E552E7CFD9FF72
:101940001200D9CFE6FFE1CFD9FF020EE12663C036
:10195000E9FF64C0EAFFEE52EFCFDFFFDFCF0BF00D
:101960000B500001795D000E7A5902E279C0DFFF69
:10197000DF500B6E0C6A0B50795D796F0C507A5901
:101980007A6F010EDB6ADF50F36E010EDBCFF4FFDE
:10199000F350F45C16E2010EDB50EA6A280FE96EA0
:1019A000020EEA22EF50E66E76C0E9FF77C0EAFF4A
:1019B000762B000E7723E552E750EF6E010EDB2AFF
:1019C000E2D7000ED8807955000E7A5528E265C01E
:1019D000E9FF66C0EAFFEE52080EEF6E65C0E9FF50
:1019E00066C0EAFF020EE926000EEA22280EEE6E1D
:1019F000020EED6E63C0E9FF64C0EAFFEF50400BDA
:101A000007E165C0E9FF66C0EAFFC80EEF6E06D0C9
:101A100065C0E9FF66C0EAFF880EEF6E28D065C09A
:101A2000E9FF66C0EAFFEE52080EEF6E65C0E9FFFF
:101A300066C0EAFF020EE926000EEA22200EEE6ED4
:101A4000020EED6E65C0E9FF66C0EAFF840EEF6E20
:101A50007B517C1107E005D07CC0FAFF00017B516F
:101A6000F96EFADF0001789F895101E1B9DD020EBC
:101A7000E15C02E2E16AE552E16EE552E7CFD9FFAF
:101A80001200D9CFE6FFE1CFD9FFE6520001738FF4
:101A9000010EE66EE66AE66A540EE66E0F0EE66E1C
:101AA0005DEC14F00B6E050EE15E0B50200EE66E41
:101AB000E66AE66A000EE66E020EE66E5DEC14F073
:101AC0000B6E050EE15E0B50648CDF6A020EDF5C6C
:101AD00010E2DF50EA6A840FE96E000EEA22EF6A34
:101AE000DF50EA6A860FE96E000EEA22EF6ADF2A0B
:101AF000EDD7010EE66EE66AE66A620EE66E000E4D
:101B0000E66E5DEC14F00B6E050EE15E0B50649C0E
:101B10000001080E6B6F020E6C6F000E636F020EF9
:101B2000646F63C065F064C066F022C261F0615109
:101B300003E1100E606F13D0010EE66EE66A610ECF
:101B4000E66E000EE66E010EE66EE66A06EC13F037
:101B50000B6E060EE15E0B500001200E606FE55229
:101B6000E552E7CFD9FF1200800E0201205D5BE154
:101B70000001C00E736F02012351030A34E0010A11
:101B80000EE0030A03E00001736B4DD00001200E4C
:101B9000716F280E726F120E746F756B44D02251E4
:101BA000F66EF76AD890F636F736B10EF626280E9E
:101BB000F7220900F5CF71F00A00F5CF72F0020E9E
:101BC0000001F76A7125F66E7251F7220800F5CF11
:101BD00074F0030EF76A7125F66E7251F722080051
:101BE000F5CF75F020D0030E225D1AE22251F66E79
:101BF000F76AD890F636F736B30EF626280EF72297
:101C00000900F5CF71F00A00F5CF72F071C0F6FF50
:101C100072C0F7FF0800F5500001746F756B02D0B9
:101C20000001736B00D01200D9CFE6FFE1CFD9FFDE
:101C3000020EE1260201286B296B20511F0B020ABC
:101C400012E0030A0DE0010A01E042D00001738FA7
:101C50000201288100017F0502E10201288338D0BA
:101C60000001738F35D00001738F020124BF10D0A3
:101C700024510F0BE96EEA6AD890E936EA36670E0E
:101C8000E926000EEA22EECFDEFFEDCFDDFF0FD01A
:101C900024510F0BE96EEA6AD890E936EA366B0EEA
:101CA000E926000EEA22EECFDEFFEDCFDDFFDECF2C
:101CB000E9FFDDCFEAFFEF50800B09E0DECFE9FF5F
:101CC000DDCFEAFFEF50040B02E0010E286F00D0D9
:101CD000000173AF07D0280E716F020E726F73810F
:101CE000020E746F020EE15C02E2E16AE552E16EFF
:101CF000E552E7CFD9FF12000F0153A115D063C001
:101D0000E9FF64C0EAFFEF5080080DE16BC0E9FF16
:101D10006CC0EAFFEF50840806E163C0E9FF64C0CD
:101D2000EAFF8C0EEF6E5391629A12006084629803
:101D300064820001010E806F000EE66EE66AE66EB8
:101D4000E66A750EE66EE66A06EC13F00B6E060E9A
:101D5000E15E0B5012000001806B000EE66EE66A39
:101D6000E66EE66A740EE66EE66A06EC13F00B6E3B
:101D7000060EE15E0B506492609462A402D06294FD
:101D8000FCD71200D9CFE6FFE1CFD9FFE652000120
:101D90002D0E886FFD0E811553E17E0E8115E840F2
:101DA0007F0B040DF3CF63F0F4CF64F0000E6327D4
:101DB000020E642363C065F064C066F0657563C09D
:101DC000E9FF64C0EAFFEF503C0BE842E8420D082F
:101DD00035E1DF6A080EDF5C23E263C0E9FF64C01F
:101DE000EAFF020EE926000EEA22EE50EFCFEAFFEC
:101DF000E96EEF50E66EDF50EA6A200FE96E020EE0
:101E0000EA22E552E750EF6E63C0E9FF64C0EAFFE3
:101E1000020EE926000EEA22EE2AEF22DF2ADAD7A6
:101E200063C0E9FF64C0EAFF020EE926000EEA2261
:101E3000200EEE6E020EED6E0DD801D03AD805D010
:101E4000FD0E8115040801E159D8E552E552E7CFAE
:101E5000D9FF120000016F6B896B8C6B8D6B836BEC
:101E6000706B6BC0E9FF6CC0EAFFEF9E6B756BC0D7
:101E7000E9FF6CC0EAFFEF9E6B7565C0E9FF66C0C5
:101E8000EAFFEF9E736B746B756B786B796B7A6B93
:101E900092D8000EE66EE66AE66EE66A030EE66E1D
:101EA000E66A06EC13F00B6E060EE15E0B50DEEFF9
:101EB0000BF0020E0001705D02E143DD1ED0706B7D
:101EC00083511AE165C0E9FF66C0EAFFEE52080ED1
:101ED000EF6E65C0E9FF66C0EAFF020EE926000E5C
:101EE000EA22200EEE6E020EED6E65C0E9FF66C0BE
:101EF000EAFF8C0EEF6E01D0836B1200D9CFE6FFA4
:101F0000E1CFD9FFE6526BC0E9FF6CC0EAFFEF50AA
:101F1000400B01E0010EDF6E00016B75080E605D85
:101F20000CE122C25CFF0F015C5104E00001100EC5
:101F3000606F03D00001040E606F700528E16BC074
:101F4000E9FF6CC0EAFF020EE926000EEA22280E25
:101F5000EE6E020EED6E93DC020E00016F5D07E186
:101F60006BC0E9FF6CC0EAFF840EEF6E0FD0DF504C
:101F700007E16BC0E9FF6CC0EAFFC80EEF6E06D048
:101F80006BC0E9FF6CC0EAFF880EEF6E0FD078AF30
:101F90000CD07B517C1107E005D07CC0FAFF00011A
:101FA0007B51F96EFADF0001789F706BE552E552C4
:101FB000E7CFD9FF120002012051600BE842E8424E
:101FC000E842E842E842000901E058D021510C0AF9
:101FD00054E00B0A43E00C0A35E0010A26E00B0A44
:101FE00022E0020A20E0030A1CE0080A10E0010ACD
:101FF0000CE00F0A08E0030A01E03FD00001738FF4
:10200000080E606F3BD0B0DD39D03BDD37D000012A
:10201000610E716F000E726F7381010E746F738F9A
:102020002DD002DE2BD02BD829D024510001716F86
:10203000726B620E7127000E72237381010E746F32
:10204000738F1CD00001738F02012451EA6A620F62
:10205000E96E000EEA2222C2EFFF10D0000EE66EFB
:10206000E66AE66EE66A020EE66EE66A06EC13F0D3
:102070000B6E060EE15E0B5001D000D01200D9CFDE
:10208000E6FFE1CFD9FF050EE1260201220510E1AE
:1020900020511F0B00090CE10001738F030E020198
:1020A000215D04E10001010E7F6F02D000017F6B12
:1020B0000201225101E020D120511F0B020801E052
:1020C0001BD124510F0B000901E116D124510F0B34
:1020D000010801E211D1200E0001605D01E00CD188
:1020E000738F020124BF1AD024510F0BE96EEA6AE4
:1020F000D890E936EA36670EE926000EEA22EECFDE
:10210000DEFFEDCFDDFF24510F0BEA6A860FE96E8B
:10211000000EEA22020EEFCFDBFF19D024510F0B85
:10212000E96EEA6AD890E936EA366B0EE926000EC7
:10213000EA22EECFDEFFEDCFDDFF24510F0BEA6A7E
:10214000840FE96E000EEA22020EEFCFDBFFD950BA
:10215000020FE96EDACFEAFFEF50010B03E1000E48
:10216000DF9401D0DF8424BF10D024510F0BE96E1F
:10217000EA6AD890E936EA36670EE926000EEA22C6
:10218000DECFEEFFDDCFEDFF0FD024510F0BE96E58
:10219000EA6AD890E936EA366B0EE926000EEA22A2
:1021A000DECFEEFFDDCFEDFF030E215D23E1DECFBD
:1021B000E9FFDDCFEAFFEF50800B13E024BF09D029
:1021C00024510F0BEA6A860FE96E000EEA22EF82B5
:1021D00008D024510F0BEA6A840FE96E000EEA2240
:1021E000EF82840E0B6EDECFE9FFDDCFEAFF0B50EE
:1021F000EF1282D0DF74DECFE9FFDDCFEAFFEF50D0
:10220000800B1BE0DECFE9FFDDCFEAFFEF9EDECFE4
:10221000E9FFDDCFEAFFEF8C020EE66EE66ADECF65
:10222000E6FFDDCFE6FF050EE66EE66A06EC13F08C
:102230000B6E060EE15E0B5005D0DECFE9FFDDCF61
:10224000EAFFEF8CDF74D950020FE96EDACFEAFFB4
:10225000EF50020B07E1DECFE9FFDDCFEAFFEF50E1
:10226000800B2DE0020124BF09D024510F0BEA6A34
:10227000860FE96E000EEA22EF9208D024510F0B70
:10228000EA6A840FE96E000EEA22EF923B0E0B6EB3
:10229000DECFE9FFDDCFEAFF0B50EF16020EE66E50
:1022A000E66ADECFE6FFDDCFE6FF050EE66EE66A04
:1022B00006EC13F00B6E060EE15E0B5008D03B0EE1
:1022C0000B6EDECFE9FFDDCFEAFF0B50EF16020108
:1022D00024510F0B0C6A530F0B6E0F0E0C22030EC2
:1022E0000BC0DBFF040E0CC0DBFF030EDBCFE9FFEE
:1022F000040EDBCFEAFFEF90050EE15C02E2E16A3B
:0C230000E552E16EE552E7CFD9FF120074
:04230C00DACFE4FF41
:10231000E2CFDAFFE9CFE4FFEACFE4FFF6CFE4FF54
:10232000F7CFE4FFF5CFE4FFF3CFE4FFF4CFE4FF12
:10233000FACFE4FF00EE00F00B0EE80403E3EECF6B
:10234000E4FFFBD700EE0BF0030EE80403E3EECF4F
:10235000E4FFFBD7E65297EC08F0E55200EE0DF0F3
:10236000030EE80403E3E5CFEDFFFBD700EE0AF030
:102370000B0EE80403E3E5CFEDFFFBD7E5CFFAFF53
:10238000E5CFF4FFE5CFF3FFE5CFF5FFE5CFF7FFAE
:10239000E5CFF6FFE5CFEAFFE5CFE9FFE5CFDAFFCE
:1023A0001100D8CFE4FFE0CFE4FFE46EDACFE4FF22
:1023B000E2CFDAFFE6529EA20AD09E9200019E2B47
:1023C000CC6A9D519E5D02E38B9001D08B80E552DB
:1023D000E5CFDAFFE550E5CFE0FFE5CFD8FF10000D
:1023E00005D8D8EC0AF022D8FED712000F0EC11281
:1023F00002D807EF08F0F00E8B1694169388290E7A
:10240000C26EC16A3E0EC06EC08E0C0ECA6ECC6A21
:10241000CB68D08EF28C9F929E929D820001986B29
:10242000996B9A6B9B6B010E9C6F120000019C5183
:1024300000E0200E0001E76E6019E8AE02D0E7343C
:1024400002D0E750605D03E36450020B01E02DD041
:1024500000019851991102E1000E08D098C0E9FFDF
:1024600099C0EAFFEF50800B01E0010E00091DE169
:10247000020130A104D08B8031C29DF003D08B903B
:1024800000019D6B400EE66E300EE66E020EE66EAB
:10249000E66A010EE66E87EC09F00B6E050EE15E52
:1024A0000B50F3CF98F0F4CF99F01200D9CFE6FF9C
:1024B000E1CFD9FF020EE126DE6ADD6AC282C2B236
:1024C000FED7C350DF6E010EC4CFDBFFDECF0BF0B3
:1024D000DDCF0CF00BC0F3FF0CC0F4FF020EE15C8B
:1024E00003E200D0E16AE552E16EE552E7CFD9FFA1
:1024F000120000019F51A01104E1100E9F6F270EE2
:10250000A06F9F07000EA05B64A20AD09F51A0118C
:1025100006E18B708BA002D08B8201D08B922ED0E3
:102520000001605103E18B908B9228D0600503E19C
:102530008B808B8223D0020E605D03E18B808B92B7
:102540001DD0040E605D03E18B908B8217D0100EBE
:10255000605D07E100019F51A01102E18B708B9239
:102560000DD0200E605D0AE100019F51A01106E12F
:102570008B708BA002D08B9201D08B821200120044
:1025800012001200120055EF13F012001E0EE66E3C
:10259000010EE66E50EC09F0E552E552400EE66E93
:1025A000300EE66E020EE66EE66A010EE66E87EC0F
:1025B00009F00B6E050EE15E0B50F3CF98F0F4CFEF
:1025C00099F0120000017F0520E1000180051DE166
:1025D000A094D6DF64920001806B0001100EA36FFF
:1025E0000E0EA46FA307000EA45BA351A411FAE181
:1025F0006484080EA36F070EA46FA307000EA45BEC
:10260000A351A411FAE16494A0841200D9CFE6FF8B
:10261000E1CFD9FFFD0EDBCF06F0FE0EDBCF07F0DA
:10262000050E061801E1075039E0E868061802E1D6
:102630007F0E071831E0030E061801E107502AE06B
:10264000020E061801E1075023E0010E061801E111
:1026500007501CE0740E061801E1075015E0750ED6
:10266000061801E107500EE0730E061801E107504D
:1026700007E0720E061801E1075001E010D00FD0FC
:1026800080DF0DD07CDF0BD07BDF09D07FDF07D070
:102690007CDF05D078DF03D075DF01D000D0010EDC
:0A26A00000D0E552E7CFD9FF120089
:0626AA00020120511F0B8C
:1026B000010801E065D0245101E062D0060E215DE1
:1026C00022E12351230A1EE0010A11E0030A01E07E
:1026D0001AD0000161050AE10001440E716F280E55
:1026E000726F090E746F756BC00E736F0CD00001A2
:1026F000950E716F280E726F1C0E746F756BC00E85
:10270000736F01D000D002012051600BE842E84213
:10271000E842E842E842010801E032D021510B0AC8
:1027200029E0080A1CE0090A14E0080A07E00B0A7D
:1027300004E0080A01E024D023D022D00001A10E39
:10274000716F000E726F010E746F756BC10E736F37
:1027500017D00001800E736F23C2A1F011D00001C9
:10276000A20E716F000E726F010E746F756B810E89
:10277000736F06D00001800E736F22C2A2F000D0EA
:02278000120045
:0E278200000EF66E100EF76E000EF86E0001DF
:102790000900F550936F0900F550946F03E19367BA
:1027A00001D03DD00900F5508E6F0900F5508F6FB4
:1027B0000900F550906F09000900F550E96E090015
:1027C000F550EA6E090009000900F550916F090003
:1027D000F550926F09000900F6CF95F0F7CF96F00B
:1027E000F8CF97F08EC0F6FF8FC0F7FF90C0F8FFCC
:1027F0000001915302E1925307E00900F550EE6E9B
:102800009107F8E29207F9D795C0F6FF96C0F7FF57
:1028100097C0F8FF00019307000E945BBFD712002A
:102820001201000200000008D804DF0502000102C6
:10283000000109022900010100C032090400000260
:1028400003000000092111010001221C000705817D
:1028500003400001070501034000010403090424AB
:10286000037500500044003700380030004300403A
:102870000067006D00610069006C002E0063006F4E
:10288000006D00120349004D0045002D0044006911
:1028900000730070000600FF0901A1011901294021
:1028A00015012540750895408100190129409100C6
:0928B000C032285B285F28832850
:0628BA00FE0EE3CFE9FF72
:1028C000FF0EE3CFEAFFE9CFF3FFEACFF4FFFB0E01
:1028D000E35003E1FC0EE35009E0FB0EE30602E2E5
:0E28E000FC0EE306FD0EE350EE6EF1D7120083
:0228EE00000EDA
:1028F000F36E00EE00F0030E01D81200EA6002D081
:0E290000EE6AFCD7F350E9601200EE6AFCD7D5
:02290E0011EEC8
:1029100000F021EE00F0F86A0A9CC1EC13F095EC8F
:0A29200014F0F0EC11F0FBD71200E8
:02292A00120099
:04292C0000000000A7
:0529300001FA000000A7
:020000040030CA
:0100000000FF
:0100010032CC
:0100020021DC
:010003001EDE
:0100050000FA
:010006008178
:0100080003F4
:01000900C036
:01000A0003F2
:01000B00E014
:01000C0003F0
:01000D0040B2
:00000001FF
